:100000000C9486000C94A3000C94A3000C94A30001
:100010000C94A3000C94A3000C94A3000C94A300D4
:100020000C94A3000C94A3000C94DC010C94FD012F
:100030000C94A3000C94A3000C94A3000C94A300B4
:100040000C94A3000C94A3000C94A3000C94A300A4
:100050000C94A3000C94A3000C94A3000C94A30094
:100060000C94A3000C94A3000C94A3000C94A30084
:100070000C94A3000C94A3000C94A3000C94A30074
:100080000C94A3000C94A3000C94A3000C94A30064
:100090000C94A3000C94A3000C94A3000C94A30054
:1000A0000C94A3000C94A3000C94A3001201000272
:1000B000FF00001001000100000101020301040320
:1000C0000904240352006500750073006300680092
:1000D000200045006C0065006B00740072006F002A
:1000E0006E0069006B00000022035500730065007C
:1000F000720020004400650076006900630065001E
:100100002000440065006D006F00000011241FBE38
:10011000CFEFDAE0DEBFCDBF11E0A0E0B1E0E0E478
:10012000FBE002C005900D92A832B107D9F711E0AB
:10013000A8E2B1E001C01D92AD32B107E1F70E9423
:10014000DC030C949E050C94000081E08093D700A2
:1001500080EA8093D80082E189BD09B400FEFDCF1A
:1001600080E98093D8001092E0001092280188E086
:100170008093E2000895E0E0F1E091E051E044E096
:1001800020812F3F09F19093E9005093EB002093D9
:10019000EC008181803811F480E40BC0803411F4CC
:1001A00080E307C0803229F0803111F080E001C087
:1001B00080E13281382B3093ED0020FF03C0109294
:1001C000F00002C04093F0009F5F33969730C1F675
:1001D0008EE78093EA001092EA0008958091D9009A
:1001E00080FD02C080E008958091E30087FD02C099
:1001F00081E0089580912801882311F083E008951B
:1002000082E008958091280108958091E80085702A
:10021000E1F30895E42FF0E02E173F0708F4422F92
:10022000262F372F7EEF9091E8009570E1F3942F01
:10023000413108F090E1F901592F09C0882311F0EC
:10024000608101C064916093F10051503196552353
:10025000A9F7290F311D491B7093E800442319F7B2
:10026000903109F308958093E90021E030E002C065
:10027000220F331F8A95E2F7EAEEF0E02083108226
:1002800008958093E9009091F3008091F200392F56
:1002900020E0280F311DC90108958093E900909155
:1002A000F300E091F200392F20E0D901AE0FB11D2B
:1002B000FD01242F352FE217F30708F49F012115C4
:1002C000310519F140E050E09091F100FB01E40F9D
:1002D000F51F90834F5F5F4F42175307A8F360915C
:1002E000F3009091F200562F40E0490F511D411547
:1002F000510559F441E050E002C0440F551F8A9562
:10030000E2F74093EA001092EA00C90108956623DB
:1003100009F11092E9002091E80020FFFCCF5091F4
:10032000F3004091F200352F20E0240F311D2115FC
:10033000310581F4FC0180E004C091919093F100BB
:100340008F5F8617D0F38091E8008E7F8093E8005E
:1003500081E0089580E008954115510559F1809399
:10036000E9008091E80080FFFCCF3091F3002091FC
:10037000F200932F80E0820F911D0097D9F480E066
:1003800090E00BC02091E80025FF06C0FB01E80FBC
:10039000F91F20812093F10001968417950790F3AF
:1003A0008091E8008E7F8093E8008FE78093E800DB
:1003B00081E0089580E008951F920F920FB60F928A
:1003C00011248F938091E1001092E10083FF0FC010
:1003D0001092E90081E08093EB001092EC0082E142
:1003E0008093ED0088E08093F000109228018F91B7
:1003F0000F900FBE0F901F9018951F920F920FB67F
:100400000F921124DF92EF92FF920F931F932F937D
:100410003F934F935F936F937F938F939F93AF938C
:10042000BF93EF93FF93DF93CF93CDB7DEB72997B9
:10043000DEBFCDBF8091F40080FF66C11092E9005D
:100440008091E80083FF5DC15091F1005983409194
:10045000F1004A838091F1009091F100392F20E062
:1004600090E0822B932B9C838B836091F1007091A1
:10047000F100372F20E070E0622B732B7E836D83B9
:100480002091F1003091F100F32FE0E030E02E2BCD
:100490003F2B38872F83E2EFE093E800463009F0E6
:1004A000BAC043E08030940709F4A3C063E0813010
:1004B000960750F471E08030970789F0A2E0803011
:1004C0009A0709F05BC110C0B3E081309B0709F4C3
:1004D00098C0E3E082309E0709F050C197C06CEAF3
:1004E00070E0FB01449189C030E0E32E31E0F32E4F
:1004F000F701DD2480E090819F3F09F081E0D80E74
:10050000339621E0E231F207A9F747E0D49E402D6F
:1005100011244E5E842F90E049870E9440048C0194
:1005200089E0D8018C9392E011969C9311974985AC
:1005300012964C93129713961C92139791E014966F
:100540009C93149715969C93159716961C92169744
:1005500090E817969C93179799E118969C93189793
:10056000F801399619968C93199784E08183128249
:100570001382D4828FEF8583168287831086DD20D5
:1005800071F1F801729691E057E035E0D7018C9156
:100590008F3FF1F050833183282F2795222727950D
:1005A000292B2283813441F0803431F0813831F0BD
:1005B000803821F083E003C081E001C082E08383C2
:1005C000D70111968C9111978483158216823796E4
:1005D0009F5F63E070E0E60EF71E9730B9F62F815B
:1005E000388581E0B8010E940A01C8010E94E20436
:1005F000C8C06EEB70E0FB01449180E00E940A01EC
:10060000C0C062EC70E0FB014491F7CF68EE70E08F
:10061000FB014491F2CF453059F42EEF2093E800CE
:100620002091E80020FFFCCF80688093E300A9C000
:10063000493081F4552309F05CC08130910509F0FF
:100640009DC081E0809328018EEF8093E8000E9496
:10065000BB0097C0483061F4503809F04AC080911F
:10066000E80080FFFCCF809128018093F1001BC03F
:100670004423D9F48091E80080FFFCCF523811F078
:1006800080E00DC06093E9008091EB0090E025E0F0
:10069000969587952A95E1F781701092E9008093ED
:1006A000F1001092F1008EEF61C0413011F0433043
:1006B00001F55230F1F40097E1F46F77862F815005
:1006C0008630B8F48EEF8093E8006093E900433001
:1006D00009F454C089E18093EB0081E090E002C00E
:1006E000880F991F6A95E2F78093EA001092EA005A
:1006F00048C0CE0101960E940D04882309F041C034
:100700003DC081E28093EB0080E090E041E2082F61
:100710000F5F2091F400019630E0082E02C035955D
:1007200027950A94E2F720FF26C00093E900209164
:10073000E80022FF1EC03091F3002091F200932FB9
:1007400080E0820F911D009769F09091F3008091F5
:10075000F200792F60E0680F711D802F0E94E00386
:100760000093E90089EF8093E8008FE78093E80029
:1007700008C04093EB008630910549F681E28093F2
:10078000EB002996DEBFCDBFCF91DF91FF91EF91B6
:10079000BF91AF919F918F917F916F915F914F9199
:1007A0003F912F911F910F91FF90EF90DF900F904D
:1007B0000FBE0F901F9018950E94A5007894FFCF50
:1007C0000F931F93DF93CF93CDB7DEB7A0970FB6EC
:1007D000F894DEBF0FBECDBF8130A1F48E010F5F54
:1007E0001F4FB80140E250E00E944D01882351F0B4
:1007F00018A2C8010E94790582E8B80140E250E0E1
:100800000E94AC01A0960FB6F894DEBF0FBECDBF1C
:10081000CF91DF911F910F910895DF93CF93CDB7C3
:10082000DEB760970FB6F894DEBF0FBECDBFAC0148
:100830009E012F5F3F4FA2E1B1E09CE00D90F901D6
:1008400001929F019150D1F71D861E861F86188A3E
:10085000FA018081833C51F48181813039F4CE01E9
:10086000019660E10E94870181E001C080E060960E
:100870000FB6F894DEBF0FBECDBFCF91DF910895C4
:10088000EF92FF920F931F93CF93DF9382309105E6
:1008900010F482E090E0C0912B01D0912C0120E077
:1008A00030E040E050E029C068817981681779071D
:1008B000D8F06817790779F48A819B812115310571
:1008C00021F0F9019383828304C090932C018093DB
:1008D0002B01DE012AC04115510519F06417750777
:1008E00018F4FE01AB01D9019E017A816B81E72EDC
:1008F000E7017E01062FF62EE7012097A9F64115A4
:100900005105F9F0481B590B4430510580F48281A0
:100910009381109729F013969C938E93129704C09D
:1009200090932C0180932B01DF01129645C0DF01CB
:10093000A40FB51F8D939D93425050405183408327
:100940003BC02091290130912A012115310541F444
:10095000209124013091250130932A01209329010F
:1009600020912601309127012115310541F42DB741
:100970003EB74091220150912301241B350BA091D9
:100980002901B0912A01A217B307A0F42A1B3B0B3F
:100990002817390778F0AC014E5F5F4F24173507F1
:1009A00048F04A0F5B1F50932A01409329018D9311
:1009B0009D9302C0A0E0B0E0CD01CDB7DEB7E6E088
:1009C0000C948F05CF93DF93009709F48FC0FC013F
:1009D00032971382128260912B0170912C01611564
:1009E000710581F420813181280F391F80912901FF
:1009F00090912A018217930761F5F0932A01E09301
:100A0000290174C0EB0180E090E0CE17DF0740F4CD
:100A10002A813B81CE012115310501F1E901F5CF94
:100A2000D383C283DF014D915D919D01240F351F5A
:100A3000C217D30761F428813981240F351F2E5F37
:100A40003F4F318320832A813B8133832283009768
:100A500029F4F0932C01E0932B0148C0DC0113969C
:100A6000FC93EE931297EC0149915991C40FD51F55
:100A7000EC17FD0779F420813181240F351F2E5F9B
:100A80003F4F11963C932E932281338113963C93D2
:100A90002E931297E0E0F0E0DB0112968D919C918D
:100AA0001397009721F0E62FF72FBC01F5CF9B019C
:100AB0002E5F3F4FDB018D919C911197820F931F09
:100AC0004091290150912A014817590779F430972C
:100AD00029F410922C0110922B0102C01382128271
:100AE0002250304030932A0120932901DF91CF9189
:100AF0000895DC016C9161566A3108F0605E6F5BAD
:100B00006D93C1F708952A88398848885F846E8478
:100B10007D848C849B84AA84B984C884DF80EE8021
:100B2000FD800C811B81AA81B981CE0FD11D0FB62A
:100B3000F894DEBF0FBECDBFED010895F894FFCF4E
:100B4000802002812002FF2002FF2002FF2002FFFE
:100B5000200256657273696F6E20312E30000000DE
:080B6000000020002D0100003F
:00000001FF
